:044000000241253222
:01400B003282
:01401300327A
:01401B003272
:01402300326A
:01402B003262
:10412500758107124121E582600302403374004422
:1041350000602974642400F974413400FA904164E4
:10414500780075A000E493F2A308B8000205A0E585
:0F41550082B501F1E583B502EC75A0FF0240339E
:1040330012405C80FEA298B3E433FA70F8C298850C
:10404300998222858299A299B3E433FA70F8C299CE
:1040530022AA8274052AF5822275985053890F4348
:104063008920758840758780758BFD758DFDC29994
:104073007582451240467582441240467582591234
:104083004046758232124046758230124046758230
:104093002012404675824D124046758241124046B9
:1040A30075822012404675824B12404675824F122C
:1040B30040467582541240467582411240467582CD
:1040C3002012404675824112404675824C1240468A
:1040D30075824912404675824B12404675824112E1
:1040E300404675820D12404675820A1240461240C0
:1040F30038E582FA8A82C002124046D0028A82C020
:1041030002124054E582D002FA8A82124046758236
:104113000D12404675820A12404602407322758290
:02412300002278
:00000001FF
